:0A1D94000001020203030404050528
:100AE200E4F55BF55AF559F558C20AC207C209C2C4
:100AF20008121C8A120C8F7E167F008E0A8F0B75CD
:100B0200121675131275081675091C7510167511D3
:100B12004A751416751578EE54E07003020C2975A7
:100B22005C00755D808E5E8F5FC374A29FFF74163A
:100B32009ECF2402CF3400FEE48F578E56F555F532
:100B420054F553F552F551F550AF57AE56AD55AC7D
:100B520054AB53AA52A951A850C31208875026E594
:100B62005D2553F582E55C3552F58374CDF0E5538E
:100B72002401F553E43552F552E43551F551E4358B
:100B820050F55080C4E4F553F552F551F550AF5786
:100B9200AE56AD55AC54AB53AA52A951A850C3128C
:100BA20008875031AE52AF53E55F2FF582E55E3EC6
:100BB200F583E0FDE55D2FF582E55C3EF583EDF022
:100BC200EF2401F553E43EF552E43551F551E43595
:100BD20050F55080B9855C0A855D0B74002480FF56
:100BE200741634FFFEC3E5139FF513E5129EF5124A
:100BF200C3E50D9FF50DE50C9EF50CC3E50F9FF5C2
:100C02000FE50E9EF50EC3E5099FF509E5089EF571
:100C120008C3E5119FF511E5109EF510C3E5159F78
:100C2200F515E5149EF514D2E843D82090E668E065
:100C32004409F090E65CE0443DF0D2AF90E680E0FB
:100C420020E105D20B121A8E90E680E054F7F053A1
:100C52008EF8C20A3008051208BEC208300A2912EC
:100C62001E295024C20A121BE320071690E682E0D6
:100C720030E704E020E1EF90E682E030E604E02095
:0D0C8200E0E4121ABD121E2B1217B980C734
:1008BE0090E6B9E0700302096F1470030209EC248C
:1008CE00FE7003020A6F24FB7003020969147003A1
:1008DE0002096314607314607624056003020ACE65
:1008EE00121E2D4003020ADA90E6BBE024FE6022BF
:1008FE0014603324FD601114602224067048E50A4A
:10090E0090E6B3F0E50B8037E51290E6B3F0E51311
:10091E00802DE50C90E6B3F0E50D8023E50E90E614
:10092E00B3F0E50F801990E6BAE0FF121AE9AA06B5
:10093E00A9077B01EA494B600DEE90E6B3F0EF900C
:10094E00E6B4F0020ADA020AD3121D3F020ADA12E4
:10095E001DE6020ADA1212BE020ADA121D2D020A70
:10096E00DA121E2F4003020ADA90E6B8E0247F6006
:10097E001514601924027063A207E43325E0FFA268
:10098E0009E4334F8041E490E740F0803F90E6BCAD
:10099E00E0547EFF7E00E0D394807C0040047D0115
:1009AE0080027D00EC4EFEED4F2494F582741D3EC8
:1009BE00F583E493FF3395E0FEEF24A1FFEE34E6DA
:1009CE008F82F583E0540190E740F0E4A3F090E6C7
:1009DE008AF090E68B7402F0020ADA020AD3121E33
:1009EE00314003020ADA90E6B8E024FE60162402D3
:1009FE006003020ADA90E6BAE0B40105C207020A01
:100A0E00DA020AD390E6BAE0705590E6BCE0547E66
:100A1E00FF7E00E0D394807C0040047D0180027D47
:100A2E0000EC4EFEED4F2494F582741D3EF583E4EA
:100A3E0093FF3395E0FEEF24A1FFEE34E68F82F5AF
:100A4E0083E054FEF090E6BCE05480131313541F61
:100A5E00FFE0540F2F90E683F0E04420F0806D808D
:100A6E0064121E33506690E6B8E024FE601924022C
:100A7E00705A90E6BAE0B40104D207804F90E6BAFD
:100A8E00E064026047803E90E6BCE0547EFF7E004C
:100A9E00E0D394807C0040047D0180027D00EC4E0A
:100AAE00FEED4F2494F582741D3EF583E493FF33DF
:100ABE0095E0FEEF24A1FFEE34E68F82F5838008E9
:100ACE00120080500790E6A0E04401F090E6A0E00E
:030ADE004480F061
:010AE10022F2
:03003300021E1793
:041E170053D8EF327B
:101C8A00758CE0758AC0E58954F04401F589758E32
:081C9A0003D28CD2A9D2AF22C3
:03000B000213B825
:1013B800C0E0C0F0C083C082C0D075D000C000C0FB
:1013C80001C002C003C004C005C006C007758CE098
:1013D800758AC0D28CE47F607EEAFDFCAB4FAA4ED2
:1013E800A94DA84CC31208875019AF4FAE4EAD4D4A
:1013F800AC4CEF2401F54FE43EF54EE43DF54DE4E9
:101408003CF54CE47F01FEFDFCAB4FAA4EA94DA86C
:101418004CC31208877008E5A054F02534F5A0E500
:101428002B2401FFE4352AFEE4FCFDAB4FAA4EA9AC
:101438004DA84CC3120887700553A0F0C28CD00782
:10144800D006D005D004D003D002D001D000D0D02F
:09145800D082D083D0F0D0E03244
:1016000012010002000000401816416900000102AA
:1016100000010A06000200000040010009022E003D
:1016200001010080FA0904000004FF000000070522
:1016300001024000000705820200020007050202C5
:101640000002000705810240000009022E0001018E
:101650000080FA0904000004FF00000007050102F1
:101660004000000705820240000007050202000258
:101670000007058102400000040309041003510023
:101680004800590043004300440020001603510065
:10169000480059002D0032003200200020002000B8
:0416A0002000000026
:100FB900608028000203010101010107000000020D
:100FC900000002001332320A080C0C08000000006D
:100FD9000000003F020302020202020700000002B1
:100FE9000000020013320A12100C0C080000000065
:100FF9000000003F0215030303030307000000027A
:10100900000002001332120A080C0C08000000004C
:101019000000003F02150303030303070000000259
:101029000000020013320A12100C0C080000000024
:101039000000003F60242887000000000000000035
:101049000000000000000000000000000000000097
:101059000000000000000000000000004728808018
:06106900000008CA4E0061
:1011580090E60174CAF090E6F574FFF0902880E0FC
:1011680090E6F3F0902881E090E6C3F0902882E0C2
:1011780090E6C1F0902883E090E6C2F0902885E0E0
:1011880090E6C0F0902886E090E6F4F075AF07741A
:1011980028F59A7400F59B759DE4E4F59EFF90E6AA
:1011A8007BE090E67CF00FBF80F490E67174FFF06E
:1011B800F5B490E672E04480F043B680000000E4A5
:1011C80090E6C4F000000090E6C5F0902887E09013
:1011D800E6C6F0902888E090E6C7F0902889E0906D
:1011E800E6C8F090288AE090E6C9F090288BE09055
:1011F800E6CAF090288CE090E6CBF090288DE0903D
:0B120800E6CCF090288EE090E6CDF0E0
:0112130022B8
:03004300021300A5
:0300530002130095
:10130000021CA200021D1700021D0100021CBA00EF
:1013100002195A0002191D00021E3500021E360075
:10132000021E3700021E38000215A50002146100DB
:10133000021E3900021E3A00021E3B00021E3C0043
:10134000021E3D00021E3600021E3E00021E3F002D
:10135000021E4000021E4100021E4200021E430007
:10136000021E4400021E3600021E3600021E360017
:10137000021E4500021E4600021E4700021E4800D3
:10138000021E4900021E4A00021E4B00021E4C00B3
:10139000021E4D00021E4E00021E4F00021E500093
:1013A000021E5100021E5200021E5300021E540073
:0813B000021E5500021E56004A
:101ABD0090E682E030E004E020E60B90E682E03034
:101ACD00E119E030E71590E680E04401F07F147EE7
:0C1ADD00001218D790E680E054FEF022C2
:101BE30090E682E044C0F090E681F0438701000074
:041BF30000000022CC
:101A8E00300B0990E680E0440AF0800790E680E093
:101A9E004408F07FDC7E051218D790E65D74FFF0E7
:0F1AAE0090E65FF05391EF90E680E054F7F0225E
:021AE900A9074B
:101AEB00AE14AF158F828E83A3E064037017AD0124
:101AFB0019ED7001228F828E83E07C002FFDEC3E6E
:091B0B00FEAF0580DF7E007F00C3
:011B140022AE
:1018D7008E688F6990E600E054187012E56924015C
:1018E700FFE43568C313F568EF13F569801590E6D3
:1018F70000E05418FFBF100BE56925E0F569E568BE
:1019070033F568E5691569AE68700215684E6005BC
:06191700121BF780EE2216
:101BF7007400F58690FDA57C05A3E582458370F901
:011C070022BA
:10106F00C1820223000002311040C100C106C10538
:0B107F00C10404480000000001400014
:081B410090E679F07F057E00BB
:101B49008E688F69E569456860177F957E00121C6C
:101B590016000000000000E569156970E715688046
:021B6900E32275
:100C8F0090E600E054E74410F000000000000090F0
:100C9F00E61074A0F000000090E60B7401F090E6EF
:100CAF001274E0F0000000E490E613F000000090F2
:100CBF00E614F000000090E615F000000090E61832
:100CCF00740CF000000090E6D27402F090E6047409
:100CDF0080F00000007402F0000000E4F00000005B
:100CEF00121158E490E671F075B4FF90E672F0754A
:100CFF00B6BF75B1FF90E670F075B2FFC28CD287A8
:100D0F00D286121D7C75230275240000000090E628
:100D1F001074A0F000000000000090E611F0000039
:100D2F000090E65EE04408F0000000E490E68DF0ED
:100D3F0090E65EE04404F0000000E490E68FF012CD
:100D4F001A5EC2A17FAA7E00121D9E75280075290A
:100D5F00B47543017544907531107532B8754606F8
:100D6F0075472C121DF6121DF690E67AE054FEF030
:100D7F00E4FD7F901219FA7F647E001218D77DFF71
:100D8F007F421219FA7F647E001218D7E4FD7F4E5E
:100D9F001219FA7535FFE4F53890E782E535F090D2
:0B0DAF00E781E538F0121E1F021CEA6D
:10173000D205E538D3940040037535FF90E678E094
:101740004480F07491121B4190E679E090E7C0125A
:101750001B4490E679E090E7C1121B4490E679E0E3
:1017600090E7C2121B4490E679E090E7C3121B4455
:1017700090E678E04440121B4490E678E04480F024
:101780007442121B4190E679E535121B4490E678CD
:10179000E04440121B4490E678E04480F090E67903
:1017A000744E121B4490E679E538121B4490E6789B
:0917B000E04440121B44C2052272
:1017B900E54B2401F54BE4354AF54AE43549F54949
:1017C900E43548F548E47FE87E03FDFCAB4BAA4AC3
:1017D900A949A848C31208877006FD7F901219FA13
:1017E9007FA07E867D017C00AB4BAA4AA949A84807
:1017F900C31208877009121E1B121730121E1F7F91
:10180900407E0D7D037C00AB4BAA4AA949A848D369
:101819001208874009E4F54BF54AF549F5483001C6
:1018290013754001E5B130E6032006F8120EC2C275
:0518390001E4F540226E
:021E2900D322C2
:021E2B00D322C0
:021E2D00D322BE
:1012BE0090E680E030E71800000090E6207402F01F
:1012CE00000000E490E621F0000000D2028016003B
:1012DE000000E490E620F000000090E6217440F05B
:0D12EE00000000C20290E6BAE0F541D322F4
:101D2D0090E740E541F0E490E68AF090E68B04F010
:021D3D00D322AF
:081DE60090E6BAE0F527D322D4
:101D3F0090E740E527F0E490E68AF090E68B04F018
:021D4F00D3229D
:021E2F00D322BC
:021E3100D322BA
:021E3300D322B8
:10008000E4F560F56190E6B9E012089800B4B300B9
:10009000F7B50241B60278C102F6C20340C503A417
:1000A000C603D9C9045ECA0492CB0521CC056BCD29
:1000B000000005F9E490E68AF090E68BF090E6A067
:1000C000E020E1F990E68BE0F560E4F5B5F5B3905A
:1000D000E60174CAF0E490E6C3F090E6C2F0D20103
:1000E00000000090E6047480F00000007402F0004C
:1000F0000000E4F00205FBE490E68AF090E68BF065
:1001000090E6A0E020E1F990E68BE0F560D3943F23
:100110004024E4F56174402561F582E434E7F58319
:10012000E0FF74AB2561F582E43428F583EFF00538
:1001300061E561B440DF7F8A7E00121D9E9028AB8E
:10014000E0FF7E00121DA79028ABE0FF7E00121D8D
:10015000B09028ABE0FF7E00121DB99028ACE0758E
:10016000F004A4FFAEF0121DC29028ACE075F004BC
:10017000A4FFAEF0121DCB9028ACE075F004A4FFF4
:10018000AEF0121DD49028B0E0C394025013902812
:10019000CCE090E6C07005744EF08016749CF08040
:1001A000119028CCE090E6C07005749FF080037435
:1001B0009DF09028CEE0F5399028CBE0F5379028D7
:1001C000CFE0F5429028D9E0F536A3E0FEA3E07C2D
:1001D000002400F526EC3EF5259028B1E0F533E546
:1001E0003370037533019028B6E0FEA3E07C002451
:1001F00000F529EC3EF528A3E0FEA3E02400F54439
:10020000EC3EF5439028B2E0FEA3E02400F532EC8A
:100210003EF531A3E0FEA3E02400F547EC3EF546B1
:100220009028BCE0FEA3E02400F53FEC3EF53E90B4
:1002300028BAE0FEA3E02400F530EC3EF52F0205DD
:10024000FBE4F56174AB2561F582E43428F583E0C5
:10025000FF74402561F582E434E7F583EFF0056132
:10026000E561B440DF000000E490E68AF0000000A1
:1002700090E68B7440020339E490E68AF090E68BB6
:10028000F090E6A0E020E1F990E68BE0F560C298FE
:10029000D3940050030205FB90E740E0940A500716
:1002A000E02430FF121D6390E740E0B40A057F614F
:1002B000121D6390E740E0B40B057F62121D63904E
:1002C000E740E0B40C057F63121D6390E740E0B4A3
:1002D0000D057F64121D6390E740E0B40E057F6555
:1002E000121D6390E740E0640F60030205FB7F6628
:1002F000121D630205FB90E74074C9F0A37403F07C
:10030000A3740CF0A37426F0A37407F0A374EEF0AA
:10031000A37401F0E4A3F0A37453F0300205E4A346
:10032000F0800690E74974FFF0000000E490E68A50
:10033000F000000090E68B740AF0121A5E0205FBD2
:1003400090E678E04480F090E6797491F07F647EE6
:1003500000121C1690E679E090E740F07F647E0082
:10036000121C1690E679E090E741F07F647E00125F
:100370001C1690E679E090E742F07F647E00121C44
:100380001690E679E090E743F090E678E04440F09C
:10039000000000E490E68AF000000090E68B740410
:1003A000F00205FBE490E68AF090E68BF090E6A080
:1003B000E020E1F990E68BE0F560D3940150030270
:1003C00005FB90E740E0FD7F4E1219FA90E741E00F
:1003D000FD7F421219FA0205FBE490E68AF090E6EE
:1003E0008BF090E6A0E020E1F990E68BE0F560D399
:1003F000940150030205FB90E740E05480C41313BE
:1004000013540124FF92A3E05440C4131354032453
:10041000FF92A2E05420C413540724FF92A1E05499
:1004200010C4540F24FF92A0A3E075F00AA4FFAEFD
:10043000F01218D790E740E05408131313541F2408
:10044000FF92A3E054041313543F24FF92A2E054FC
:1004500002C31324FF92A1E01392A00205FB90E6D1
:10046000BCE0756200F5632005FDAD6390E6BEE07B
:10047000FB7EE77567E77568407FA0121C2DAD63B2
:1004800090E6BEE0FB7EE77567E77568407FA002F7
:100490000552E490E68AF090E68BF090E6A0E0202A
:1004A000E1F990E6BCE0D3940750030205FB200578
:1004B000FD78EB7C287D017B017AE679BC7E007FAC
:1004C000011206CD90E6BEE0FF7E0078EC7C287D30
:1004D000017B017AE779401206CD90E6BEE004FD8B
:1004E0007A287BEB7F50121C6E78EB7C287D017B99
:1004F000017AE679BC7E007F011206CD90E6BEE06F
:10050000FF7E0078EC7C287D017B017AE779401240
:1005100006CD90E6BEE004FD7A287BEB7F50020515
:10052000F490E6BCE0756200F5632005FDAD6390D4
:10053000E6BEE0FB7EE77567E77568407FA2121CA8
:100540002DAD6390E6BEE0FB7EE77567E77568401A
:100550007FA2121C2DE490E68AF000000090E6BE17
:10056000E090E68BF00000000205FBE490E68AF0E4
:1005700090E68BF090E6A0E020E1F990E6BCE0D3B5
:10058000940740772005FD78EB7C287D017B017A7C
:10059000E679BC7E007F011206CD90E6BEE0FF7ECC
:1005A0000078EC7C287D017B017AE779401206CD4A
:1005B00090E6BEE004FD7A287BEB7F51121C6E783A
:1005C000EB7C287D017B017AE679BC7E007F0112FD
:1005D00006CD90E6BEE0FF7E0078EC7C287D017BB6
:1005E000017AE779401206CD90E6BEE004FD7A2854
:0C05F0007BEB7F51121C6E8002D322C3F3
:0105FC0022DC
:101CA200C0E0C083C082D2085391EF90E65D740118
:081CB200F0D082D083D0E032B3
:101D0100C0E0C083C0825391EF90E65D7404F0D0CF
:061D110082D083D0E03215
:101D1700C0E0C083C0825391EF90E65D7402F0D0BB
:061D270082D083D0E032FF
:10195A00C0E0C083C08285100C85110D850D82857B
:10196A000C83A37402F085080E85090F850F828502
:10197A000E83A37407F05391EF90E65D7410F0D0D4
:06198A0082D083D0E032A0
:101CBA00C0E0C083C082D20A5391EF90E65D7408F7
:081CCA00F0D082D083D0E0329B
:10191D00C0E0C083C08290E680E030E72085080CEF
:10192D0085090D850D82850C83A37402F085100E3B
:10193D0085110F850F82850E83A37407F05391EFE8
:0D194D0090E65D7420F0D082D083D0E032AF
:011E3500327A
:011E36003279
:011E37003278
:011E38003277
:1015A500C0E0C0F0C083C082C0D075D000C000C00C
:1015B50001C002C003C004C005C006C007C2AF1207
:1015C5001E1B00000090E68F7404F000000053918C
:1015D500EF90E65FE04404F0121E1FD2AFD007D0B3
:1015E50006D005D004D003D002D001D000D0D0D091
:0815F50082D083D0F0D0E03277
:10146100C0E0C083C082C0D075D000C004C006C037
:011471000773
:10147200C2AF90E6A1E020E1F990E780E0146016A7
:1014820024F86020240C60481460491460501470E1
:1014920052752200804D90E782E0F53590E781E0B9
:1014A200F538803FD28C90E781E0540FF534A3E009
:1014B200FEA3E07C002400FFEC3EC313F52AEF13E9
:1014C200F52B754F00754E00754D00754C0080135D
:1014D200C28C800F90E781E024FF9206800575227E
:1014E20000D20300000090E68DE4F05391EF90E605
:0714F2005FE04408F0D2AFF7
:0F14F900D007D006D004D0D0D082D083D0E0323C
:011E39003276
:011E3A003275
:011E3B003274
:011E3C003273
:011E3D003272
:011E3E003271
:011E3F003270
:011E4000326F
:011E4100326E
:011E4200326D
:011E4300326C
:011E4400326B
:011E4500326A
:011E46003269
:011E47003268
:011E48003267
:011E49003266
:011E4A003265
:011E4B003264
:011E4C003263
:011E4D003262
:011E4E003261
:011E4F003260
:011E5000325F
:011E5100325E
:011E5200325D
:011E5300325C
:011E5400325B
:011E5500325A
:011E56003259
:061214008F648C658D66FD
:10121A0053640753A0BF121C12E4F567F568C37440
:10122A00029568FFE564A807088002C313D8FC305A
:10123A00E00543A020800353A0DF121C1243A01034
:10124A00121C1253A0EF121C120568E56870020501
:10125A0067C39403E5676480948040C2E4F567F548
:10126A0068C374099568FFE566AE65A80708800536
:10127A00CEC313CE13D8F930E00543A02080035320
:10128A00A0DF121C1243A010121C1253A0EF121C52
:10129A00120568E56870020567C3940AE567648009
:1012AA00948040BD43A040121C1253A0BF7F0A7E07
:0412BA0000021C16FC
:091D9E00AD07AC06E4FF021214CB
:091DA700AD07AC067F0402121422
:091DB000AD07AC067F0502121418
:091DB900AD07AC067F060212140E
:091DC200AD07AC067F010212140A
:091DCB00AD07AC067F0202121400
:091DD400AD07AC067F03021214F6
:1019FA008D64AD0790E678E04480F090E679EDF0EA
:101A0A007F647E00121C1690E679E564F07F647E9E
:101A1A0000121C1690E678E04440F07F647E0002D3
:021A2A001C1688
:0E1C08007F0A7E00121C16121E237F0A7E0029
:101C1600EF7803C333CE33CED8F9FFEF4E6007EF2C
:071C26001F70F81E80F5227B
:0315FD00C2802287
:031E2300D2802248
:0512FB00C283D2842231
:051DFE00D283D2842213
:051E0300C283C284222D
:051E0800C282D281221C
:051E0D00C282C2812227
:051E1200D282D2812202
:031E2600C2852250
:091D7000121DFE121E23121E12A8
:031D7900D28522EE
:0C1D7C00121D79121E081212FB0215FD48
:101CD2001215FD121E12121E26121DFE121E0812CF
:081CE2001E231212FB021D7902
:10188B001215FD121C12121E0D121C12121E031227
:10189B001C08121E08121C121212FB121C1212151B
:1018AB00FD121C12121E12121C12121E26121C12D8
:1018BB00121DFE121C12121E08121C081212FB1211
:0C18CB001C12121D797F0A7E00021C1600
:101D5100E4FFFE121CD20FBF00010EBE0BF5BF1631
:011D6100F28F
:011D6200225E
:0C1D8800C2867F647E00121C16D28622E8
:101A5E0053B17FE4F564F56543B1807F1E7E0012BD
:101A6E0018D753B17F7F1E7E001218D70565E56526
:0F1A7E0070020564C39405E5646480948040D9C8
:011A8D002236
:041E1B0043B180222D
:041E1F0053B17F221A
:091DDD007F4F121D6343B1202267
:081DEE0053B1DF7F43021D63C6
:10108B00E4FFFEE53BFDE4FCFB7A01F9F81207DF18
:10109B00E4FB7A01F9F81207DF8F2CE4FFE53CFE45
:1010AB00E4FDFCFB7A01F9F81207DF8F2EE53DFF1B
:1010BB008F2D121D70E530452F7003121D88E537FB
:1010CB00B40102C287121DDDE539706D752201E591
:1010DB002C75F040A485F066F567AF227E00AC66F8
:1010EB00AD67120742D3EF9400EE940040147FC417
:1010FB007E03121B49121730E567156770DC156606
:10110B0080D8756600852E67AF227E00AC66AD6712
:10111B00120742D3EF9400EE940040147FC47E007C
:10112B00121B49121730E567156770DC156680D8FE
:10113B00AF2D7E001218D78009752201E5226401BC
:0C114B0060FA121DEEE537B40102D287F5
:011157002275
:101B1500AD07AC06D3ED9400EC9400401E00000028
:101B2500EE90E6D0F0000000ED90E6D1F000000068
:0C1B350075BB04000000E5BB30E7FB229C
:02183E00AC06F6
:1018400090E6C0E0FBE490E618F090E6C0744EF03D
:10185000EC90E6D0F0000000EF90E6D1F000000040
:1018600075BB04000000E5BB30E7FB90E604748024
:10187000F00000007402F0000000E4F000000090AE
:0A188000E618740CF090E6C0EBF0DF
:01188A00223B
:101B6B00AD07AC06000000ED25E0EC3390E6D0F0BD
:101B7B00000000ED25E090E6D1F000000075BB04FD
:091B8B00000000E5BB30E7FB227D
:101508009028AEE0FFE4FCFDFEFB7A01F9F8120733
:1015180054C004C005C006C0079028ADE0FFE4FC35
:10152800FDFEFBFA7901F8120754D003D002D0016E
:10153800D000EF2BFBEE3AFAED39F9EC38F89028A9
:10154800AFE0FFE4FCFDFEEB2FF53DEE3AF53CED98
:1015580039F53BEC38F53AE47F18AB3DAA3CA93B9A
:10156800A83AD31208874026E53D24E8F53DE53C36
:1015780034FFF53CE53B34FFF53BE53A34FFF53AFB
:1015880012108BE530452F7011121D51800CE5307B
:0D159800452F7003121D5112108B02188B8D
:100EC200121E1FC203754002121508754003121E3E
:100ED2001B300303020FB8E4F562F563C3E56395C3
:100EE20029E56295285029E4F564F565C3E5659521
:100EF200337480F8656498500D121CD20565E5655F
:100F020070EA056480E60563E56370D0056280CC13
:100F1200E536D39400400EAF367E00AC31AD3212CE
:100F2200074212183ED3E5269400E52594004007B7
:100F3200AF26AE25121B6BE4F560F561C3E5619542
:100F420047E5609546502C121B94E4F564F565C3A1
:100F5200E56595337480F8656498500D121CD205CE
:100F620065E56570EA056480E60561E56170CD05B9
:100F72006080C9E4F562F563C3E5639544E5629573
:100F8200435029E4F564F565C3E56595337480F84B
:100F9200656498500D121CD20565E56570EA05641A
:100FA20080E60563E56370D0056280CC121D70AFE8
:060FB2003FAE3E121B15CC
:010FB8002216
:101B9400000000E53225E0E5313390E6D0F00000A6
:101BA40000E53225E090E6D1F000000075BB0400AA
:081BB4000000E5BB30E7FB2255
:101CEA00E490E608F075C83443985053877FC2AC35
:071CFA0075CBFF75CA6422DF
:0D1D6300309902C2998F993099FDC29922E2
:101BBC0090000020981CA3AF82AE83E4FCFD7BFA5E
:101BCC007AFFF9F8C31208715004D2008004C200E5
:061BDC0080E1C298AF9900
:011BE20022E0
:041C2D008F648B66CF
:101C310090290BEDF0E564C313FF7A297B0B7D013D
:101C4100121C6EE564C313FFAB68AA67AD66021C84
:011C51005240
:081DF600E4F51BD2E9D2AF2293
:1019900090E678E020E6F9C2E990E678E04480F04D
:1019A000EF25E090E679F090E678E030E0F990E617
:1019B00078E04440F090E678E020E6F990E678E0C0
:0619C00030E1D6D2E9225D
:101A2C00A90790E678E020E6F9E51B702390E678AC
:101A3C00E04480F0E925E090E679F08D16AF03A93B
:101A4C00077517018A188919E4F51A751B01D32239
:021A5C00C322A3
:1019C600A90790E678E020E6F9E51B702590E67811
:1019D600E04480F0E925E0440190E679F08D16AF09
:1019E60003A9077517018A188919E4F51A751B03E7
:0419F600D322C32213
:03004B00020DBAE9
:100DBA00C0E0C083C082C085C084C086758600C07A
:100DCA00D075D000C000C001C002C003C006C00771
:100DDA0090E678E030E206751B06020EA490E678EB
:100DEA00E020E10CE51B64026006751B07020EA4F5
:100DFA00E51B24FE605F14603624FE7003020E9524
:100E0A0024FC7003020EA124086003020EA4AB178F
:100E1A00AA18A919AF1A051A8F827583001206F348
:100E2A0090E679F0E51A65167070751B05806B906F
:100E3A00E679E0AB17AA18A919AE1A8E8275830053
:100E4A00120720751B02E5166401704E90E678E0E1
:100E5A004420F08045E51624FEB51A0790E678E0AE
:100E6A004420F0E51614B51A0A90E678E04440F0FA
:100E7A00751B0090E679E0AB17AA18A919AE1A8E6D
:100E8A0082758300120720051A800F90E678E044E5
:100E9A0040F0751B008003751B005391DFD007D00B
:100EAA0006D003D002D001D000D0D0D086D084D0D2
:080EBA0085D082D083D0E03224
:101C52001219C6E51B24FA600E146006240770F3FD
:0C1C6200D322E4F51BD322E4F51BD322AF
:101C6E00121A2CE51B24FA600E146006240770F37A
:0C1C7E00D322E4F51BD322E4F51BD32293
:030000000216A441
:0C16A400787FE4F6D8FD7581690216EB32
:1005FD00E709F608DFFA8046E709F208DFFA803EE0
:10060D0088828C83E709F0A3DFFA8032E309F608CC
:10061D00DFFA8078E309F208DFFA807088828C8334
:10062D00E309F0A3DFFA806489828A83E0A3F608E8
:10063D00DFFA805889828A83E0A3F208DFFA804CC2
:10064D0080D280FA80C680D4806980F28033801099
:10065D0080A680EA809A80A880DA80E280CA803302
:10066D0089828A83ECFAE493A3C8C582C8CCC5837A
:10067D00CCF0A3C8C582C8CCC583CCDFE9DEE7804A
:10068D000D89828A83E493A3F608DFF9ECFAA9F0C9
:10069D00EDFB2289828A83ECFAE0A3C8C582C8CC1F
:1006AD00C583CCF0A3C8C582C8CCC583CCDFEADE38
:1006BD00E880DB89828A83E493A3F208DFF980CC9A
:1006CD0088F0EF60010E4E60C388F0ED2402B40493
:1006DD000050B9F582EB2402B4040050AF2323453A
:0606ED00822390064D730C
:1006F300BB010CE58229F582E5833AF583E02250BC
:1007030006E92582F8E622BBFE06E92582F8E22205
:0D071300E58229F582E5833AF583E493221F
:10072000F8BB010DE58229F582E5833AF583E8F00F
:10073000225006E92582C8F622BBFE05E92582C8BB
:02074000F222A3
:10074200EF8DF0A4A8F0CF8CF0A428CE8DF0A42ECB
:02075200FE2285
:10075400E88FF0A4CC8BF0A42CFCE98EF0A42CFC44
:100764008AF0EDA42CFCEA8EF0A4CDA8F08BF0A4C2
:100774002DCC3825F0FDE98FF0A42CCD35F0FCEB21
:100784008EF0A4FEA9F0EB8FF0A4CFC5F02ECD39E6
:0F079400FEE43CFCEAA42DCE35F0FDE43CFC2253
:1007A30075F008758200EF2FFFEE33FECD33CDCC0D
:1007B30033CCC58233C5829BED9AEC99E582984090
:1007C3000CF582EE9BFEED9AFDEC99FC0FD5F0D66D
:1007D300E4CEFBE4CDFAE4CCF9A88222B800C1B997
:1007E3000059BA002DEC8BF084CFCECDFCE5F0CBD5
:1007F300F97818EF2FFFEE33FEED33FDEC33FCEB0E
:1008030033FB10D703994004EB99FB0FD8E5E4F9C8
:10081300FA227818EF2FFFEE33FEED33FDEC33FCB5
:10082300C933C910D7059BE99A4007EC9BFCE99AA9
:10083300F90FD8E0E4C9FAE4CCFB2275F010EF2FEE
:10084300FFEE33FEED33FDCC33CCC833C810D707EE
:100853009BEC9AE899400AED9BFDEC9AFCE899F829
:0E0863000FD5F0DAE4CDFBE4CCFAE4C8F922BC
:10087100EB9FF5F0EA9E42F0E99D42F0EC6480C8FE
:0608810064809845F0229E
:10088700EB9FF5F0EA9E42F0E99D42F0E89C45F0C7
:01089700223E
:10089800D083D082F8E4937012740193700DA3A3EF
:1008A80093F8740193F5828883E473740293686003
:0608B800EFA3A3A380DF03
:1016B000020AE2E493A3F8E493A34003F68001F264
:1016C00008DFF48029E493A3F85407240CC8C3333B
:1016D000C4540F4420C8834004F456800146F6DF0A
:1016E000E4800B0102040810204080900FB9E47ED2
:1016F000019360BCA3FF543F30E509541FFEE493FF
:10170000A360010ECF54C025E060A840B8E493A3C5
:10171000FAE493A3F8E493A3C8C582C8CAC583CAF0
:10172000F0A3C8C582C8CAC583CADFE9DEE780BEA8
:01108A000065
:00000001FF
